:020000040000FA
:100000000128850107309F00031383163A308500CD
:1000100003138312860107309F0003138316FF30FA
:10002000860007308100031383120608A0001230F7
:10003000A10001308A0020080021003E0319642835
:10004000A20002308A0020080022A30003308A00A8
:1000500020080023A70004308A0020080024A800FC
:1000600005308A0020080025A90006308A002008F3
:100070000026A4008030A5009230A6008513051349
:100080000514051024087820250878202608043E49
:1000900078200514051021087820220878202308EC
:1000A00078200514051027087820280878202908CA
:1000B00078200514051024087820250878202608C3
:1000C0007820051405106328031383160730810078
:1000D0000313831205156F2005116F206A2807305E
:1000E000AA0081010B110B1D7328AA0B71280800AF
:1000F000AB000830AC00AB0D031C8513031885174B
:0C01000005170513AC03031908007B2849
:04010C000034003487
:1002000082073C343C343E3400343C340034003407
:1002100000343C343C343C3400343C343C34003412
:1002200000343C34433443343C3400340034003430
:1002300000343C343C343C343C340034003400342E
:1002400000342D343C34433443340034003400341F
:1002500000343C343C343C343C340034003400340E
:1002600000343C34433443343C34003400340034F0
:1002700000343C343C343C343C34003400340034EE
:1002800000343C343C343C343C34003400340034DE
:10029000003443343C3443344334003400340034B9
:1002A00000343C343C343C343C34003400340034BE
:1002B00000343C34433443343C34003400340034A0
:1002C00000343C343C343C343C340034003400349E
:1002D00000343C343C343C343E340034003400348C
:1002E00000343B34003400343B34003400340034F8
:1002F00000343C343C343C343C343C340034003432
:1003000000343C343C343C343C343C340034003421
:1003100000343C343C343C343C343C340034003411
:1003200000343C343C343C343C343C340034003401
:1003300000343C343C343C343C343C3400340034F1
:1003400000343C343C343C343C343C3400340034E1
:1003500000343C3400343C343C343C34003400340D
:1003600000343C3400343C343C343C3400340034FD
:1003700000343C3400343C343C343C3400340034ED
:1003800000343C3400343C343C343C3400340034DD
:1003900000343C34003443344334433400340034B8
:1003A00000343C34003443343C343C3400340034B6
:1003B000003400340034003400340034003400349D
:1003C000003400340034003400340034003400348D
:1003D000003400340034003400340034003400347D
:1003E000003400340034003400340034003400346D
:1003F000003400340034003400340034003400345D
:100400008207003400348034003400340034003477
:10041000003400340034003400340034003400343C
:10042000003400348034803400340034003400342C
:10043000003400340034003400340034003400341C
:10044000003400340034803480340034003400340C
:1004500000340034003400340034003400340034FC
:1004600000340034803480340034003400340034EC
:1004700000340034003400340034003400340034DC
:1004800000340034003400340034003400340034CC
:10049000003480340034803480340034003400343C
:1004A00000340034003400340034003400340034AC
:1004B000003400348034803400340034003400349C
:1004C000003400340034003400340034003400348C
:1004D00000340034003400348034003400340034FC
:1004E00000346034003400346034003400340034AC
:1004F000003400340034003400340034003400345C
:10050000003400340034003400340034003400344B
:10051000003400340034003400340034003400343B
:10052000003400340034003400340034003400342B
:10053000003400340034003400340034003400341B
:10054000003400340034003400340034003400340B
:1005500000340034003400340034003400340034FB
:1005600000340034003400340034003400340034EB
:1005700000340034003400340034003400340034DB
:1005800000340034003400340034003400340034CB
:1005900000343C34003480348034803400340034FF
:1005A000003400340034803400340034003400342B
:1005B000003400340034003400340034003400349B
:1005C000003400340034003400340034003400348B
:1005D000003400340034003400340034003400347B
:1005E000003400340034003400340034003400346B
:1005F000003400340034003400340034003400345B
:1006000082070334023402340034023400340034EC
:10061000003402340234043400340434043400342A
:100620000034023403340334023400340034003420
:100630000034023402340234013400340034003413
:1006400000340434053403340534003400340034F9
:1006500000340234043404340334003400340034ED
:1006600000340534033403340534003400340034DA
:1006700000340234023402340134003400340034D3
:1006800000340634033403340234003400340034BC
:1006900000340234023402340234003400340034B2
:1006A000003403340334033402340034003400349F
:1006B0000034023402340234013400340034003493
:1006C0000034023402340234023400340034003482
:1006D0000034023402340234023400340034003472
:1006E0000034023400340034023400340034003466
:1006F000003404340234023404340234003400344C
:10070000003402340234023402340234003400343F
:10071000003402340234053402340234003400342C
:10072000003402340234023402340234003400341F
:10073000003402340234023402340234003400340F
:1007400000340234023402340234023400340034FF
:1007500000340234003402340234023400340034F1
:1007600000340234003402340234023400340034E1
:1007700000340234003402340234023400340034D1
:1007800000340334003403340334033400340034BD
:1007900000340334003403340334033400340034AD
:1007A00000340234003402340234023400340034A1
:1007B0000034003400340034003400340034003499
:1007C0000034003400340034003400340034003489
:1007D0000034003400340034003400340034003479
:1007E0000034003400340034003400340034003469
:1007F0000034003400340034003400340034003459
:1008000082070C34B834713400345E340034003460
:10081000003440343F347D340034F334DD3400346C
:100820000034D03429342934703400340034003496
:1008300000341C341B341B34D434003400340034F2
:1008400000343F34A9342F3487340034003400346A
:1008500000342034F434E834B0340034003400344C
:100860000034F034563456342F340034003400341D
:1008700000343A3439343934F2340034003400343A
:100880000034B834DC34D834E63400340034003476
:10089000003462341E3462342C34003400340034AA
:1008A00000343C343B343B34F43400340034003402
:1008B000003428346C346C34F834003400340034A0
:1008C0000034B234B634B2348E34003400340034E0
:1008D0000034BE34BD34BD34B5340034003400348B
:1008E00000342B34003400340F340034003400342E
:1008F0000034ED3476347634C9342F340034003487
:1009000000347F347E347E346D3437340034003428
:10091000003484348434073478343C340034003474
:100920000034EB34EA34EA34E234C73400340034BF
:100930000034EF34EF34EF34E634CB340034003499
:100940000034DD34DD34DD34D934CB3400340034CC
:1009500000345034003450344E34473400340034C2
:1009600000345034003450344E344D3400340034AC
:1009700000345C3400345C345A3453340034003472
:100980000034B9340034B934B734B03400340034EE
:100990000034B9340034B934B734B03400340034DE
:1009A00000347B340034CB347A3475340034003472
:1009B0000034003400340034003400340034003497
:1009C0000034003400340034003400340034003487
:1009D0000034003400340034003400340034003477
:1009E0000034003400340034003400340034003467
:1009F0000034003400340034003400340034003457
:100A000082070134013401340034013400340034ED
:100A10000034013481348134003481348134003431
:100A200000340134A1344134013400340034003442
:100A300000340134C13481340134003400340034D2
:100A40000034813481344134813400340034003442
:100A50000034013441348134013400340034003432
:100A600000340134A1344134813400340034003482
:100A700000340134C134843401340034003400348F
:100A800000348134C1348134813400340034003482
:100A90000034813481342134813400340034003412
:100AA00000340134C1348134013400340034003462
:100AB00000340134D134A134013400340034003422
:100AC0000034813421344134813400340034003422
:100AD00000340134E134C134C13400340034003412
:100AE0000034C13400340034413400340034003464
:100AF00000348134F134E134813401340034003481
:100B000000340134F134E134013401340034003470
:100B10000034213411348134213421340034003440
:100B200000340134F934F134013401340034003438
:100B300000348134793471348134813400340034A8
:100B4000003481347D34793401348134003400340C
:100B50000034713400346D34313471340034003475
:100B60000034E1340034DD34A134E13400340034A5
:100B700000345934003455341934593400340034B5
:100B80000034F5340034F134B534F5340034003435
:100B90000034F5340034F134B534F5340034003425
:100BA0000034F934003475347934F93400340034C5
:100BB0000034003400340034003400340034003495
:100BC0000034003400340034003400340034003485
:100BD0000034003400340034003400340034003475
:100BE0000034003400340034003400340034003465
:100BF0000034003400340034003400340034003455
:100C00008207C334C334C3340034C33400340034E3
:100C10000034C334C3348334003483348334003425
:100C20000034C334C334C334C33400340034003418
:100C30000034C334C334C334C33400340034003408
:100C4000003483348334C3348334003400340034B8
:100C50000034C334833483348334003400340034A8
:100C600000348334C334C334833400340034003458
:100C70000034C334C334C334C334003400340034C8
:100C800000348334C334C334833400340034003438
:100C90000034C334C334C334C334003400340034A8
:100CA0000034C334C334C334C33400340034003498
:100CB0000034C334C334C334C33400340034003488
:100CC0000034C334C334C334C33400340034003478
:100CD0000034C334C334C334C33400340034003468
:100CE0000034C33400340034C334003400340034DE
:100CF00000348334C334C3348334C3340034003405
:100D00000034C334C334C334C334C3340034003474
:100D10000034C334C3348334C334C33400340034A4
:100D20000034C334C334C334C334C3340034003454
:100D30000034C334C334C334C334C3340034003444
:100D40000034C334C334C334C334C3340034003434
:100D50000034C3340034C334C334C33400340034E7
:100D60000034C3340034C334C334C33400340034D7
:100D70000034C3340034C334C334C33400340034C7
:100D80000034C3340034C334C334C33400340034B7
:100D90000034C3340034C334C334C33400340034A7
:100DA0000034C3340034C334C334C3340034003497
:100DB0000034003400340034003400340034003493
:100DC0000034003400340034003400340034003483
:100DD0000034003400340034003400340034003473
:100DE0000034003400340034003400340034003463
:100DF0000034003400340034003400340034003453
:02400E00303F41
:00000001FF
